:100000001AC091C0A7C030C02FC02EC02DC02CC0B8
:100010002BC02AC029C028C027C027C025C024C0A3
:1000200023C022C021C0E2C0F1C00CC120C12EC13A
:1000300049C164C17DC111241FBECFEDCDBF10E009
:10004000A0E6B0E0ECE6F3E002C005900D92A23627
:10005000B107D9F720E0A2E6B0E001C01D92A836B2
:10006000B207E1F785D080C1CBCF1F920F920FB6B8
:100070000F9211248F939F93AF93BF93809164004D
:1000800090916500A0916600B09167000196A11D56
:10009000B11D8093640090936500A0936600B093B7
:1000A00067008091640090916500A0916600B09116
:1000B0006700892B8A2B8B2B59F48FEF9FEFDC0184
:1000C0008093640090936500A0936600B0936700EE
:1000D000809163008823F1F080916000909161002D
:1000E00001969093610080936000809160009091F0
:1000F0006100892B31F48FEF9FEF90936100809323
:1001000060008091600090916100069710F4959ACC
:1001100001C09598BF91AF919F918F910F900FBEA5
:100120000F901F9018951F920F920FB60F921124E7
:100130008F9380916300833021F08091630082303F
:1001400019F481E0809363008F910F900FBE0F90A0
:100150001F9018951F920F920FB60F9211241092B4
:100160006100109260000F900FBE0F901F901895C5
:100170008E9A8D9A8C9A969A959A949AC09AC19AC8
:10018000B99AC29ABA9AC39ABB9ABC9AC49A82E0A4
:1001900080BF83E083BF8CE786BF81E089BF85B7DE
:1001A000826085BF8BB780648BBF85B7846085BF55
:1001B0008BB780688BBF78941092640010926500B2
:1001C00010926600109267001092630081E097E041
:1001D00026E035E044E053E062E0E0916300F0E0C7
:1001E000E830F105D0F7ED5EFF4F0994C090640050
:1001F000D0906500E0906600F090670078E8C71640
:1002000073E1D706E104F10440F3ABC0C19AC29A8E
:10021000C39A969AC4989498E0916000F091610016
:100220003697D8F6B099D9CFC49A949A9698609395
:1002300063001092640010926500109266001092A4
:100240006700CBCFC0906400D0906500E09066005E
:10025000F090670077EEC7167DE0D706E104F10461
:1002600008F4BBCFC498C29850936300B6CFB09B3C
:10027000B4CFC198969A10926400109265001092C3
:1002800066001092670040936300A7CFC09064009F
:10029000D0906500E0906600F090670072E8C716A5
:1002A00076E0D706E104F10408F497CFC3981092E2
:1002B00064001092650010926600109267003093FF
:1002C00063008BCFC0906400D0906500E090660022
:1002D000F090670073EAC71671E0D706E104F104F5
:1002E00008F47BCFC29A10926400109265001092BD
:1002F000660010926700209363006FCFC090640087
:10030000D0906500E0906600F090670076E7C71631
:1003100072E0D706E104F10458F0C19A109264002B
:10032000109265001092660010926700909363002F
:10033000C0906400D0906500E0906600F090670087
:1003400079E9C71676E0D706E104F10408F445CF51
:10035000C39A109264001092650010926600109289
:0C03600067008093630039CFF894FFCF52
:02036C00060089
:00000001FF
